:20FFD600A269E000E000E000E000E000E000E000E000E000E000E000E000FD00E000E000C3
:0AFFF600E000E000E000E000E000A1
:20C00000464C094B5420202020005350454349414C50524F472E3F20202000535045432E07
:20C0200050524F47204B4C41523F200050524F4752414D46454C00000000000000414E475A
:20C0400045204B4F443A00000000000000007300204E31202020204E32202020204E332030
:20C0600000492F4F20544553543F00494E47084E4720414B542E3A00555447084E47204189
:20C080004B542E3A0046454C484953544F52494B3F2020202000414E542E50524F472E3AE5
:20C0A000000050554D505449443A0000000044524946545241444552494E47202121205488
:20C0C000454D502031204F46465345543A0054454D502032204F46465345543A0073656B20
:20C0E000006D003F002E0050524F4752414D4D4552494E4720202000202000DF4320006D3D
:20C10000696E00204D4544202000205554414E200050002000300025006800094E4452413F
:20C12000204B4F443A0000000000000042525954205354520A4D4D454E000000004D415256
:20C140004B45524120494E53502E3F20200053540A545449443A000000000000000000563F
:20C1600009524D455220534B0A4C4A54414E4B004752414E554C4154004449534B415220B8
:20C18000202000534B0A4C4A4552202000564944415245203D2053544152542020004645B9
:20C1A0004C20485556520A52454C53452020005354094E4720485556454E20460A5220003C
:20C1C000202020202020202020202020202020200056415454454E46594C4C4E494E47200A
:20C1E000200046594C4C45522056415454454E2020200044524946544B4C415220202020DC
:20C200002020200046454C2046594C4C4E494E47202020200050524F562050524F475241B2
:20C220004D202020200046454C204859445241554C494B202020002020202053544F505017
:20C24000414420202020200046454C204B4C094D534B5944442020200046454C2053094B58
:20C260004552482E4E495608200046454C204B4F5247445249564E494E470046454C2053C7
:20C28000094B4252595441524520200046454C204D4F544F52534B59444420200046454CD3
:20C2A000200A482D534B594444202020200046454C2056415454454E545259434B20005317
:20C2C000544152543D4A412C203F3D4E454A20004C41444441205354414E444152443F2070
:20C2E000004C41444441205354414E444152443F3F00414E54414C2050524F4752414D3A17
:20C30000000000204449534B544944202000000000000000094E445241200A5652494741E0
:20C320002020200000534B0A4C4A54454D503A000000000000004449534B54454D503A0054
:20C340000000000000000053455041524154494F4E3A000000000000534B0A4C4A5449448E
:20C360003A00000000000000004E495608204449534B3A000000000000004E4956082053A1
:20C380004B0A4C4A3A000000000000464C094B54205449443A00000000000000534B0A4C0F
:20C3A0004A4D4544454C000000000000004B4C4152200A56524947412020202020005052BD
:20C3C0004F4752414D4D2E204B4C41523F200053414B4E41522032342056444320210045FA
:20C3E0004E474C4953483F202020202020202000444555545343483F2020202020202020EA
:20C40000004652414E434149533F20202020202020005356454E534B413F2020202020209C
:20C4200020200053554F4D493F20202020202020202020004E454445524C414E44533F2071
:20C4400020202020004954414C49414E4F3F20202020202020004E4F52534B3F20202020A0
:20C4600020202020202000455350414E4F4C3F20202020202020200044414E534B3F2020BB
:09C48000202020202020202000B3
:20C4A00046414E202020202020005350454349414C2050524F472E3F202000535045432E88
:20C4C0002050524F472E204F4B3F200050524F4752414D204552524F5200000000494E5014
:20C4E000555420434F44453A0000000000007300204E31202020204E32202020204E3320EB
:20C5000000492F4F20544553543F00494E47084E4720414B542E3A00555447084E472041E4
:20C520004B542E3A004552524F52204D455353414745532020004E4F2E50524F473A000075
:20C54000000050554D5054494D453A00000044524946545241444552494E47202121205495
:20C56000454D502031204F46465345543A0054454D502032204F46465345543A0073656383
:20C58000006D003F002E0050524F4752414D4D494E47202020202000202000DF4320006DEF
:20C5A000696E002057495448200020572F4F202000500020003000250068004348414E4765
:20C5C0004520434F44453A00000000005455524E204D414348494E45204F4646004D415268
:20C5E0004B20494E5350454354494F4E3F00494D50554C53452D54494D453A000000004898
:20C60000454154494E4720424F494C45522020004752414E554C45530057415348455320F9
:20C6200020200052494E53455320202000434F4E54494E5545203D2053544152540045527F
:20C64000524F5220484F4F444D4F56454D2E00434C4F534520484F4F4420464F52202000E4
:20C66000202020202020202020202020202020200057415445522D46494C4C494E472020C5
:20C68000200046494C4C53205741544552202020202000524541445920544F205741534832
:20C6A000202020004552524F522046494C4C494E4720202000545249414C2050524F4752E5
:20C6C000414D4D4520004552524F52204859445241554C494353002020494E54455252550F
:20C6E00050544544202020004552524F5220484F4F44534146455459004552524F52205310
:20C70000414645204C4556454C004552524F52205241434B204452495645004552524F52C6
:20C720002053414645545953572E20004552524F52204D4F544F5250524F5420004552528C
:20C740004F522053555045524850524F54004552524F5220574154455250524553530053EF
:20C76000544152543D5945532020203F3D4E4F004C4F4144204445462E56414C5545533F8B
:20C78000004C4F4144204445462E56414C5545533F004E4F2E204F462050524F4752533A96
:20C7A000000000205741534854494D4520000000000000004348414E4745204F54482E56A2
:20C7C000414C3F200052494E53452D54454D503A000000000000574153482D54454D503A7F
:20C7E0000000000000000053455041524154494F4E3A00000000000052494E53452D5449BE
:20C800004D453A0000000000004C4556454C20574153483A0000000000004C4556454C20AF
:20C82000424F494C45523A0000000046414E54494D453A00000000000000000052494E5387
:20C84000452D4147454E5400000000000046494E4953484544204F54482E56414C005052EF
:20C860004F47522E2046494E495348454420004D495353494E472032342056444320004516
:20C880004E474C4953483F202020202020202000444555545343483F202020202020202045
:20C8A000004652414E434149533F20202020202020005356454E534B413F202020202020F8
:20C8C00020200053554F4D493F20202020202020202020004E454445524C414E44533F20CD
:20C8E00020202020004954414C49414E4F3F20202020202020004E4F52534B3F20202020FC
:20C9000020202020202000455350414E4F4C3F20202020202020200044414E534B3F202016
:09C920002020202020202020000E
:20C940004C0E46544552202020005350455A49414C2050524F472E3F2020005350455A2E5F
:20C9600050524F472E204F4B3F20200050524F4752414D4D204645484C45520000434F4407
:20C98000452045494E474542454E3A0000007300204E31202020204E32202020204E332088
:20C9A00000492F4F20544553543F00494E47084E4720414B542E3A00555447084E47204140
:20C9C0004B542E3A004645484C45524D454C44554E47454E2000414E5A2E50524F472E3A24
:20C9E000000050554D504544415545523A0044524946545241444552494E4720212120546A
:20CA0000454D502031204F46465345543A0054454D502032204F46465345543A0053656BF6
:20CA2000006D003F002E0050524F4752414D4D494552554E47202000202000DF4320004DDE
:20CA4000696E00204D4954202000204F484E452000500020003000250068004E455545529F
:20CA600020434F44453A0000000000005354524F4D2041425354454C4C454E0000494E5308
:20CA8000502E204D41524B4945522E3F2000494D50554C5344415545523A00000000004893
:20CAA0004549545A5420424F494C4552202020004752414E554C41540053500E4C454E209B
:20CAC0002020004B4C415253500E4C2000574549544552203D205354415254202000464529
:20CAE000484C2E4841554245424557472E20004841554245205343484C49455353454E0026
:20CB00002020202020202020202020202020202000460E5220574153534552460E4C4C4549
:20CB20004E00460E4C4C54205741535345522020202000424554524945425342455245493B
:20CB4000542020004645484C455220460E4C4C454E20202000564552535543482050524F5B
:20CB60004752414D4D004645484C2E4859445241554C494B2020002050524F4752414D4D82
:20CB800053544F50502020004645484C2E4B4C454D4D53434855545A004645484C2E534932
:20CBA00043482E4E4956454155004648454C2E4B4F5242414E5452494542004645484C2E27
:20CBC000534943482E534348414C54004645484C2E204D4F544F525343482E200046454844
:20CBE0004C200E482D53434855545A2020004645484C2E574153534552445255434B005337
:20CC0000544152543D4A4120203F3D4E45494E005745524B5357455254204C4144454E3F9A
:20CC2000005745524B5357455254204C4144454E3F00414E5A2E2050524F4752414D4D3A8D
:20CC40000000002053500E4C5A4549542000000000000000414E442E574552544520094E5C
:20CC600044524E3F004B4C415253500E4C544D503A000000000053500E4C54454D503A00D2
:20CC80000000000000000041425452454E4E44415545523A000000004B4C415253500E4CB8
:20CCA000444155523A000000004E49562E2053500E4C454E3A00000000004E49562E20428C
:20CCC0004F494C45523A00000000004C0E4654455244415545523A00000000004B4C41523F
:20CCE00053502E4D49544C000000000000414E44455245205745525445204F4B3F0050523C
:20CD00004F4752414D2E204645525449473F004F484E4520323420564443202020200045DD
:20CD20004E474C4953483F202020202020202000444555545343483F2020202020202020A0
:20CD4000004652414E434149533F20202020202020005356454E534B413F20202020202053
:20CD600020200053554F4D493F20202020202020202020004E454445524C414E44533F2028
:20CD800020202020004954414C49414E4F3F20202020202020004E4F52534B3F2020202057
:20CDA00020202020202000455350414E4F4C3F20202020202020200044414E534B3F202072
:09CDC0002020202020202020006A
:20CDE00056454E54494C4552200050524F472E205350454349414C453F200050524F472E19
:20CE000020535045432E204F4B3F200050524F4752414D4D452045525245555200494E53F7
:20CE20004552455220434F44453A000000007300204E31202020204E32202020204E33201C
:20CE400000492F4F20544553543F00494E47084E4720414B542E3A00555447084E4720419B
:20CE60004B542E3A00414646495343482E2045525245555220004E425245205047522E3ADC
:20CE800000004455520B4520504D503A000044524946545241444552494E47202121205475
:20CEA000454D502031204F46465345543A0054454D502032204F46465345543A007365633A
:20CEC000006D003F002E0050524F4752414D4D4154494F4E20202000202000DF4320006D49
:20CEE000696E00204156454320002053414E532000500020003000250068004E4F555645CD
:20CF0000415520434F44453A00000000455441494E445245204D4143482E000000504F496B
:20CF20004E54204420494E53504543542E0054454D505320494D50554C533A000000004D7D
:20CF4000495345200D2054454D5020424F552E004752414E554C4553004C41564520202050
:20CF600020200052494E43452020202000434F4E54494E5545203D20535441525400455279
:20CF8000522E4645524D2E4341504F542020004645524D2E204341504F5420504F555200AD
:20CFA000202020202020202020202020202020200052454D504C495353414745204541553A
:20CFC000200052454D504C49542045415520202020200050520C5445204155204C41564138
:20CFE000474520004552524555522052454D504C4953532E005047522E20455850455249EF
:20D000004D454E5420004552522E204859445241554C495155450020202020204152520CA7
:20D0200054202020202020004552522E4341504F5420534543555220004552522E4E495688
:20D04000454155205345435552004552522E454E54522E50414E49455220004552522E4996
:20D060004E54455252205345435552004552522E5345435552204D4F544555520045525205
:20D080002E20534555522053555243482E004552522E2050524553532045415520200053DE
:20D0A000544152543D4F554920203F3D4E4F4E0056414C2E4445462E205553494E453F2053
:20D0C0000056414C2E4445462E205553494E453F3F004E4252452044452050524F47522E78
:20D0E0003A0000204455522E4C41562E20000000000000004348414E47452041555452206A
:20D1000056414C3F00544D502052494E0F4147453A000000000054454D50204C415641471C
:20D12000453A00000000004455522E20534550415241543A000000004455522E2052494ECB
:20D140000F4147453A000000004E49562E204C41564147453A00000000004E49562E204217
:20D160004F55494C4C3A00000000004455522E56454E54494C2E3A00000000004147454E82
:20D18000542052494E0F2E00000000000050520C54204155545245533F202020200050529E
:20D1A0004F47522E5445524D494E0B453F20004D414E5155452044452032345644430045C3
:20D1C0004E474C4953483F202020202020202000444555545343483F2020202020202020FC
:20D1E000004652414E434149533F20202020202020005356454E534B413F202020202020AF
:20D2000020200053554F4D493F20202020202020202020004E454445524C414E44533F2083
:20D2200020202020004954414C49414E4F3F20202020202020004E4F52534B3F20202020B2
:20D2400020202020202000455350414E4F4C3F20202020202020200044414E534B3F2020CD
:09D26000202020202020202000C5
:20D28000505548414C4C494E20004552494B4F49534F484A2E3F20202020004F484A454CBB
:20D2A0004D4F494E5449204F4B3F20004F484A454C4D4156495248452000000000414E4E0A
:20D2C00041204B4F4F44493A0000000000007300204E31202020204E32202020204E33200A
:20D2E00000492F4F20544553543F00494E47084E4720414B542E3A00555447084E472041F7
:20D300004B542E3A0056494B41484953544F52494120202020004F484A454C2E4C4B4D3A3A
:20D32000000050554D50505541494B3A000044524946545241444552494E4720212120545C
:20D34000454D502031204F46465345543A0054454D502032204F46465345543A0073656B8D
:20D36000006D003F002E004F484A454C4D4F494E5449202020202000202000DF4320004D22
:20D38000494E00202B2020202000202D2020202000500020003000250068005641494844C5
:20D3A00041204B4F4F44493A000000004B41544B414953452056495254410000004B495283
:20D3C0004A41205441524B49535455533F004B09594E4E4953545953494B413A000000485D
:20D3E000555548542E564544454E204C094D4D005241455045535520005045535520202066
:20D400002020004855554854454C5520004A41544B41203D205354415254202020005649C3
:20D42000524845204B5556554E4C494B45200053554C4A45204B5550552020202020200067
:20D440002020202020202020202020202020202000564544454E54095954540A2020202072
:20D46000200054095954090920564554540920202020004B095954540A56414C4D49532039
:20D480002020200056090952092054095954540A20202020004B4F454F484A454C4D412062
:20D4A0002020202020005649524845204859445241554C2E2020005649524845205059530D
:20D4C00009595445545459005649524845204B5556554E52414A41200056495248452054E9
:20D4E0005552564152414A412000564952484520504553554B4F52492020005649524845E2
:20D500002054555256414B59544B2E005649524845204D4F4F54544F52492020005649529C
:20D52000484520594C494B55554D2E202000564952484520564553495041494E45200053EB
:20D54000544152543D202B2020203F3D202D20004C415441412056414B494F3F2020202003
:20D56000004C415441412056414B494F3F3F202020004F484A454C4D49454E204C4B4D3AF7
:20D58000000000502D41494B413A000000000000000000004D55555441204D555554203F68
:20D5A000202020200048555548542E4C094D503A000000000000504553554C094D500A5476
:20D5C0003A00000000000052454B45455420504F49533A000000000048555548542E414976
:20D5E0004B413A000000000000414E5455524920504553553A0000000000414E5455524928
:20D600002048555548543A00000000505548414C4C2E41494B413A000000000048555548A4
:20D62000542E41494E453A0000000000004D5555542056414C4D49533F20202020004F4884
:20D640004A454C4D412056414C4D49533F200056495248452032345644432021202000456F
:20D660004E474C4953483F202020202020202000444555545343483F202020202020202057
:20D68000004652414E434149533F20202020202020005356454E534B413F2020202020200A
:20D6A00020200053554F4D493F20202020202020202020004E454445524C414E44533F20DF
:20D6C00020202020004954414C49414E4F3F20202020202020004E4F52534B3F202020200E
:20D6E00020202020202000455350414E4F4C3F20202020202020200044414E534B3F202029
:09D7000020202020202020200020
:20D7100056454E54494C41542000535045432E50524F472E5354414E443F00535045432EA1
:20D730002050524F472E204F4B3F200050524F4752414D4D4120464F55540000005741435B
:20D750004854574F4F52443A0000000000007300204E31202020204E32202020204E332025
:20D7700000492F4F20544553543F00494E47084E4720414B542E3A00555447084E47204162
:20D790004B542E3A00464F5554204D454C44494E47454E20200041414E542E50524F473A7D
:20D7B0000000504F4D5054494A443A00000044524946545241444552494E4720212120541D
:20D7D000454D502031204F46465345543A0054454D502032204F46465345543A0073656301
:20D7F000006D003F002E0050524F4752414D4D4552454E2020202000202000DF4320004D61
:20D81000494E00204D4554202000204745454E2000500020003000250068004E4945555707
:20D830002E5741434854573A00000000484F4F4644534348414B2E2055495400004E415A9F
:20D85000494348542050554E543F20202000494D504F4C532054494A443A000000000056DB
:20D870004552572E20424F494C455220202020004B4F5252454C53200057415353454E20EC
:20D890002020004E4153504F454C202000564552444552203D205354415254202000464F3E
:20D8B000555420484F4544534C554954202000534C55495420484F4544202020202020000D
:20D8D0002020202020202020202020202020202000564F4F522056554C4C454E202020207C
:20D8F000200056554C54205741544552202020202020004B4C415220562E205741535345D9
:20D910004E202000464F55542056554C202020202020202000544553542050524F475241E9
:20D930004D4D41202000464F5554204F4C49455359535445454D0050524F47522E4F4E4472
:20D95000455242524F4B2E00464F5554204B4E454C42455645494C2000464F55542057416F
:20D970005445524E495645415500464F5554204B4F5246414E44522E202000464F55542063
:20D9900044455552534348414B202000504F4D50204F56455242454C415354200044524F45
:20D9B0004F474B4F4F4B20424556202020004C4147452057415445524452554B20200053AB
:20D9D000544152543D4A412020203F3D4E454500464142522E494E5354454C4C2E3F20206F
:20D9F00000464142522E494E5354454C4C2E3F3F200041414E542E50524F4752414D2E3A15
:20DA10000000002057415354494A443A2000000000000000414E44455245204745472E573F
:20DA3000494A5A3F004E4153504F4C54454D503A00000000000057415354454D503A000012
:20DA5000000000000000004E412057415353454E3A000000000000004E4153504F4C544992
:20DA70004A443A0000000000004E49562E2057415354414E4B3A000000004E49562E2042C3
:20DA90004F494C45523A000000000056454E542E2054494A443A0000000000004E4153509F
:20DAB0004F454C4D49442E000000000000414E44455245204745472E204F4B3F20005052E3
:20DAD0004F4752414D2E4B4C4141523F2020004745454E2032342056444320212020004540
:20DAF0004E474C4953483F202020202020202000444555545343483F2020202020202020C3
:20DB1000004652414E434149533F20202020202020005356454E534B413F20202020202075
:20DB300020200053554F4D493F20202020202020202020004E454445524C414E44533F204A
:20DB500020202020004954414C49414E4F3F20202020202020004E4F52534B3F2020202079
:20DB700020202020202000455350414E4F4C3F20202020202020200044414E534B3F202094
:09DB90002020202020202020008C
:208DE00056454E544F4C4120200050524F47522E205350454349414C453F0046494E45207B
:208E000050524F472E535045432E3F004552524F52452050524F4752414D4D4100434F44E9
:208E200049434520494E5055543A000000007300204E31202020204E32202020204E332044
:208E400000492F4F20544553543F00494E47084E4720414B542E3A00555447084E472041DB
:208E60004B542E3A004552524F524520202020202020202020004E522E505247523A000099
:208E800000004F524520504F4D50413A000044524946545241444552494E4720212120547A
:208EA000454D502031204F46465345543A0054454D502032204F46465345543A007365637A
:208EC000006D003F002E0050524F4752414D4D415A494F4E45202000202000DF4320004D7E
:208EE000494E0020434F4E2020002053454E5320005000200030002500680043414D424999
:208F00004120434F442E3A0000000000535045474E49204D41434348494E410000535049AC
:208F20004120434F4E54524F4C4C4F3F2000542E204420494D50554C534F3A0000000052FA
:208F4000495343414C444920424F494C455220004752414E554C4920004C41564120202065
:208F600020200053434941435155412000434F4E54494E554F203D20535441525400455236
:208F8000522E4D4F56494D204341505520200043484955444920434150552050455220001A
:208FA00020202020202020202020202020202020005249454D50494D2E20414351554120C5
:208FC00020005249454D504945204143515541202020004F4B204C4156414747494F202037
:208FE000202020004552524F5245204C4956454C4C4F20200050524F4752414D4D412050B5
:20900000524F564120004552522E2049445241554C494341202000202020204152524553F6
:20902000544F2020202020004552522E205345435552204341504F20004552522E204C4905
:20904000562E2053494355522E004552522E4D4F542E43455354454C4C4F004552522E20F1
:209060004D4943524F20504F525441004552522E2050524F54455A2E4D4F542E0045525280
:209080002E2053555252495343414C442E004552522E2050524553532E41435155410053A8
:2090A000544152543D5349202020203F3D4E4F0050524F4752414D4120424153453F2020F0
:2090C0000050524F4752414D4120424153453F3F20004E522E2050524F4752414D4D493A88
:2090E000000000204455522E4C41563A20000000000000005641522E20414C5452492056D1
:20910000414C3F200054DF20534349414351554F3A000000000054DF204C41564147474930
:209120004F3A00000000004455522E205345504152415A3A000000004455522E53434941E4
:209140004351554F3A000000004C49562E4C4156414747494F3A000000004C49562E204285
:209160004F494C45523A00000000004455522E56454E54494C2E3A00000000004252494CBE
:209180004C49414E542020000000000000414C54524920564F4C4F5249204F4B3F00464918
:2091A0004E452050524F4752414D4D413F200053454E532032342056444320212020004575
:2091C0004E474C4953483F202020202020202000444555545343483F20202020202020203C
:2091E000004652414E434149533F20202020202020005356454E534B413F202020202020EF
:2092000020200053554F4D493F20202020202020202020004E454445524C414E44533F20C3
:2092200020202020004954414C49414E4F3F20202020202020004E4F52534B3F20202020F2
:2092400020202020202000455350414E4F4C3F20202020202020200044414E534B3F20200D
:0992600020202020202020200005
:20800000564946544520202020005350455349414C50524F472E3F20202000535045432EF3
:2080200050524F472E4B4C41523F200050524F4752414D4645494C2020202020004B4F449B
:20804000453A0000000000000000000000007300204E31202020204E32202020204E33206E
:2080600000492F4F20544553543F00494E47084E4720414B542E3A00555447084E472041C9
:208080004B542E3A004645494C484953544F52494B2020202000414E542E50524F472E3A1B
:2080A000000050554D50455449443A00000044524946545241444552494E47202121205483
:2080C000454D502031204F46465345543A0054454D502032204F46465345543A0073656B60
:2080E000006D003F002E0050524F4752414D4D4552494E4720202000202000DF4320006D7D
:20810000696E00204D4544202000205554454E200050002000300025006800454E4452453B
:20812000204B4F44453A0000000000004252595420535452304D4D454E000000004D455227
:208140004B20494E53502E3F202020202000494D50554C535449443A000000000000005622
:2081600041524D455220534B594C4C54414E4B004752414E554C4154005641534B45522061
:20818000202000534B594C4C4552202000564944455245203D2053544152542020004645A4
:2081A000494C2048455454454245562E2020004C554B4B2048455454454E20464F522000FF
:2081C000202020202020202020202020202020200056414E4E46594C4C4E494E47202020A9
:2081E000200046594C4C45522056414E4E2020202020004452494654534B4C415220202048
:20820000202020004645494C204D45442046594C4C494E47005445535450524F4752414D5B
:208220002020202020004645494C204859445241554C2E202020002020202053544F5050A1
:2082400045542020202020004645494C204B4C454D4245534B2E2020004645494C2053490D
:208260004B4B45482E4E495620004645494C204B5552564452562E202020004645494C205E
:2082800053494B4B2E425259542E20004645494C204D4F544F525645524E202000464549CF
:2082A0004C20542E4B2E53494B522E2020004645494C2056414E4E545259434B202000531D
:2082C000544152543D4A412020203F3D4E4549005354442E20564552444945523F202020FA
:2082E000005354442E20564552444945523F3F202000414E54414C4C2050524F4752414D82
:208300003A0000205641534B5449443A2000000000000000454E44524520414E4E45543F50
:208320002020202000534B594C4C4554454D503A0000000000005641534B4554454D503A8F
:2083400000000000000000534550455241534A4F4E3A000000000000534B594C4C45544978
:20836000443A000000000000004E495641205641534B3A000000000000004E495641205321
:208380004B594C4C3A00000000000056494654455449443A0000000000000000544F525287
:2083A000454D494444454C0000000000004F2E4B2E20414E4E45543F2020202020005052BC
:2083C0004F4752414D204F2E4B2E3F202020004D414E474C45522032342056444320004584
:2083E0004E474C4953483F202020202020202000444555545343483F20202020202020202A
:20840000004652414E434149533F20202020202020005356454E534B413F202020202020DC
:2084200020200053554F4D493F20202020202020202020004E454445524C414E44533F20B1
:2084400020202020004954414C49414E4F3F20202020202020004E4F52534B3F20202020E0
:2084600020202020202000455350414E4F4C3F20202020202020200044414E534B3F2020FB
:09848000202020202020202000F3
:2084A00056454E54494C4152200050524F472E2045535045432E3F2020200050524F472E0E
:2084C0002045535045432E204F4B3F004552524F522050524F4752414D41202000494E54B7
:2084E000524F20434F4449474F3A000000007300204E31202020204E32202020204E332099
:2085000000492F4F20544553543F00494E47084E4720414B542E3A00555447084E47204124
:208520004B542E3A004D414E53414A4553204552524F522020004E522E505247523A0000B5
:2085400000004455522E424F4D42413A000044524946545241444552494E472021212054CC
:20856000454D502031204F46465345543A0054454D502032204F46465345543A00736563C3
:20858000006D003F002E0050524F4752414D4D4143494F4E20202000202000DF4320006DE3
:2085A000696E0020434F4E2020002053494E2020005000200030002500680043414D4249D1
:2085C0004520434F442E3A0000000000415041474152204D415155494E410000004D415240
:2085E00043415220494E53504543432E3F004455522E20494D50554C534F3A000000004334
:20860000414C454E54414E444F20424F494C52004752414E554C4F20004C4156414E444FEF
:2086200020200041434C415241444F2000434F4E54494E5541523D2053544152540045526E
:20864000522E4D4F56494D204341504F544100434552524152204341504F54412020200043
:20866000202020202020202020202020202020200050415241204C4C454E415220414755FB
:208680004100434F4749454E444F2041475541202020005055454445204C4156415220206A
:2086A000202020004552524F52204C4C454E41444F2020200050524F4752414D412044454F
:2086C0002054455354004552522E204859445241554C49434120002020494E544552555096
:2086E00043494F4E202020004552522E5345435552204341504F5441004552522E4E49567C
:20870000454C2053454755522E004552522E4D4F562E43414E4153544120004552522E5338
:20872000454E532E20505545525441004552522E204D4F544F522D50524F542E00455252E3
:208740002E50524F5445432E5445524D2E004552522E50524553494F4E20414755410053C2
:20876000544152543D53492020203F3D4E4F4E00204441544F5320464142524943413F201C
:2087800000204441544F5320464142524943413F3F004E522E2050524F4752414D413A0037
:2087A000000000204455522E4C41563A20000000000000002043414D422E4F54524F53202B
:2087C00056414C3F0054DF2041434C415241444F3A000000000054DF204C415641444F3A6F
:2087E0000000000000000053455041524143494F4E3A0000000000004455522E41434C4130
:208800005241444F3A000000004E49562E2054414E5155453A00000000004E49562E204238
:208820004F494C45523A00000000004455522E56454E54494C2E3A000000000050524F44FB
:208840002E204252494C4C4F0000000000204F54524F2056414C2E204F4B3F2020002046D2
:20886000494E414C2050524F4752414D413F0053494E2032342056444320212020200045C9
:208880004E474C4953483F202020202020202000444555545343483F202020202020202085
:2088A000004652414E434149533F20202020202020005356454E534B413F20202020202038
:2088C00020200053554F4D493F20202020202020202020004E454445524C414E44533F200D
:2088E00020202020004954414C49414E4F3F20202020202020004E4F52534B3F202020203C
:2089000020202020202000455350414E4F4C3F20202020202020200044414E534B3F202056
:098920002020202020202020004E
:2089400056454E54494C415420005350454349414C50524F472E3F20202000535045432E31
:2089600050524F47204B4C41523F200050524F4752414D46454A4C2020202020004B4F445F
:20898000453A0000000000000000000000007300204E31202020204E32202020204E332025
:2089A00000492F4F20544553543F00494E47084E4720414B542E3A00555447084E47204180
:2089C0004B542E3A0046454A4C484953544F52494B3F20202000414E542E50524F472E3AB2
:2089E000000050554D50455449443A00000044524946545241444552494E4720212120543A
:208A0000454D502031204F46465345543A0054454D502032204F46465345543A0073656B16
:208A2000006D003F002E0050524F4752414D4D4552494E4720202000202000DF4320006D33
:208A4000696E00204D4544202000205544454E20005000200030002500680041454E445206
:208A600045204B4F44453A0000000000534C554B20535452304D4D454E000000004D41529F
:208A80004B455220494E53502E3F20202000494D50554C535449443A000000000000005682
:208AA00041524D455220534B594C4C54414E4B004752414E554C4154005641534B45522018
:208AC000202000534B594C4C4552202000564944455245203D20535441525420200046455B
:208AE0004A4C204841455454454245562E20004C554B4B204845415454454E20464F520073
:208B0000202020202020202020202020202020200056414E44500846594C444E494E472059
:208B20002000500846594C4445522056414E4E2020200044524946544B4C41522020202021
:208B40002020200046454A4C204D2E2046594C444E494E47005445535450524F4752414D26
:208B600020202020200046454A4C204859445241554C494B2020002020202053544F505011
:208B8000455420202020200046454A4C204B4C454D4245534B2E20200046454A4C205349C2
:208BA0004B4B4552482E4E49560046454A4C204B555256454452455620200046454A4C20A5
:208BC0004430524B4F4E54414B54200046454A4C204D4F544F52564145524E200046454A50
:208BE0004C20542E4B2E53494B522E20200046454A4C2056414E445452594B202020005300
:208C0000544152543D4A412020203F3D4E454A005354442E20564552444945523F202020AF
:208C2000005354442E20564552444945523F3F202000414E54414C2050524F4752414D3A4A
:208C4000000000205641534B4554443A200000000000000041454E44524520305652494751
:208C6000413F202000534B594C4C4554454D503A0000000000005641534B4554454D503A06
:208C80000000000000000053455041524154494F4E3A000000000000534B594C4C45544933
:208CA000443A000000000000004E4956454155205641534B3A00000000004E495645415517
:208CC00020534B594C3A000000000056454E54494C2E5449443A00000000000054305252B4
:208CE000454D494444454C0000000000004B4C4152203056524947453F2020202000505228
:208D00004F4752414D204F2E4B2E3F202020005341564E4552203234205644432021004550
:208D20004E474C4953483F202020202020202000444555545343483F2020202020202020E0
:208D4000004652414E434149533F20202020202020005356454E534B413F20202020202093
:208D600020200053554F4D493F20202020202020202020004E454445524C414E44533F2068
:208D800020202020004954414C49414E4F3F20202020202020004E4F52534B3F2020202097
:208DA00020202020202000455350414E4F4C3F20202020202020200044414E534B3F2020B2
:098DC000202020202020202000AA
:20FF000001010A141E28323C46505152535455565758595A0001010A141E28323C3D3E3F92
:20FF200040414243444546000A141E28323C000A0F14191E23282D32373C0000010F14195C
:18FF40001E23282D3C4B5AFF000000010300010600000300000000FF26
:20FD0000DD69DF6B18DF6DBDED0B2706860197002014BDED102706860297002009BDED15CD
:20FD2000270486039700BDED9C260ABDED722605BDEC9D2003BDEC2E132B02107F0038BDB7
:20FD4000ED0B2608BDED102603152B02132B400B7C00569656810F2E0D20177A0056965653
:20FD600081002702200C132B4005152B402003142B40132B011086AFBDA2587C00689668EB
:20FD800081072E07200E7F0068200901152B0186A0BDA258132A20037C0039132A40037C38
:20FDA000003A132A10037C00387C003F860A913F2E3313288005DE3308DF337C0055142990
:20FDC000107C00357C00377C00427C0043132A8007DC3BC30001DD3B7C00367F003F132ACE
:20FDE00002037C0054964027087A00402603152904964127087A004126031529088640B757
:0AFE00001025DC69DE6B18DE6D3B97
:20E000008600B710248693B710397F10358683B71026863CB710098E00FF8600B760018679
:20E02000FFB760008604B760018600B760038600B760028604B7600318CE03E8BD9C33BD2B
:20E040009C33BDA2467F002CB6102FCE1000C6051F2E20FCB6102F81C0270A81C6270B8139
:20E06000C3270C200D142C012008142C022003142C045A26DB86F0BDA258BDF83E861497BF
:20E08000BA7F000D7F00207F0021BDF930BDF2F2BDF83EBDF9EEBDEB64BDEB36BDEEC8B6CA
:20E0A000103181FF27037EE0BCBDEEFAB6103281FF27037EE0BCBDF83E7EA15D860097036B
:20E0C000BD9C68BDED2C2700BDED1027061529407EA0007EE2FD152941BD9C68CCC096BD83
:20E0E000F042DC1ABDEF49BD9C73CCC0A2BDF042DC1CBDEF49CCC119BDF042BD9D8D122778
:20E1000001F9122704F5BD9C68B6B7159767B6B71497669707CCC0BFBDF1A09766CEB71447
:20E12000BD9D5A96679707CCC0CEBDF1A09767CEB715BD9D5A18CE01F4BD9C33BD9C68BDB7
:20E140009C73CCC050BDF0428681BD9C89BDEDA89606BDEF2CCCC113BDF0428687BD9C89B8
:20E16000BDEDE09606BDEF2CCCC113BDF042868DBD9C89BDEE189606BDEF2CCCC113BDF099
:20E1800042BDE749962D27037EE693BDED10262520B6BD9C68CCC061BDF042BD9C73CCC29A
:20E1A000BFBDF042BD9D8D1227010A122704067E9B1B7EE295142B01BD9C7ECCC085BDF045
:20E1C00042BD9C73CCC2BFBDF042BD9D8D122701E1122704DDBD9C7ECCC1C0BDF042BD9C6D
:20E1E0007ECEB7E0A600BDEF2CCCC0E5BDF042CEB7E0A601BDEF2CCCC0E5BDF042CEB7E0B5
:20E20000A602BDEF2CCCC0E5BDF042CEB7E0A603BDEF2CCCC0E5BDF042CEB7E0A604BDEF1D
:20E220002CBD9D8DBD9C7ECCC1C0BDF042BD9C7ECEB7E0A605BDEF2CCCC0E5BDF042CEB714
:20E24000E0A606BDEF2CCCC0E5BDF042CEB7E0A607BDEF2CCCC0E5BDF042CEB7E0A608BDE0
:20E26000EF2CCCC0E5BDF042CEB7E0A609BDEF2CBD9D8DBD9C7ECCC1C0BDF042BD9C7ECC9A
:20E28000C13DBDF042BD9D8D12270109122704058663BDF3E5BD9C68CCC215BDF042BD9CFB
:20E2A00073CCC2BFBDF042BD9D8D122701081227040486019703BD9C7ECCC1C0BDF042BD54
:20E2C0009C7ECCC14EBDF0429602BDEF2CBD9D8D1227020F7C0002861591022ED9860097E9
:20E2E0000220D3BD9C7ECCC01BBDF042BD9D8D12270107122704037EF5D37EE0D6860097BD
:20E3000001BDF9EE142940BDF83EBD9C68960E972E960F972FBDED2C260CBD9C68CCC3CF2C
:20E32000BDF0427EE721152903152901BDEA4D962D27037EE693BDEDA82646152930BD9C8B
:20E3400068CCC1AFBDF042BD9C73CCC1D1BDF042BD9D8D122701F9BDEABF8602912D27D64E
:20E360008601912D27C3142930BD9C68BD9C73CCC1E2BDF042142932BDE9A48601912D27F1
:20E38000A814290386019720142930BD9C73CCC1F3BDF042BD9D8D122701F91227040D7ECD
:20E3A000E3CBBDEA4D962D27227EE721BDED32260DBDEABF962D27037EE6937EE38BBDEA3D
:20E3C0004D962D27037EE6937EE38B152B80142930BD9C73CCC1C0BDF042BD9C73CCC11181
:20E3E000BDF04296208100272D9620BDEF2CCCC113BDF042BDE6D59657BDEF2CCCC0FFBD01
:20E40000F042CCC113BDF04296308100270BCCC170BDF0422003BD9C73BD9D8D12270413B0
:20E420001227022E7C0020961091202C9E860197202098BDED32260DBDEABF962D27037EE0
:20E44000E6937EE3CBBDEA4D962D27037EE6937EE3CB4F91202600BD9C73CCC1C0BDF042E5
:20E46000142930142B80BDE6D5BDEC887F00337F0034142880BDE749962D27037EE693CC09
:20E4800000091A93332EEEBDEABF962D27037EE693BDE9A4962D27037EE3CBCC000BDD33E3
:20E4A000BDEC6918CE03E8BD9C33BDEC4318CE07D0BD9C33BDEC51960281002720C60A3D51
:20E4C000188FBD9C33BDE749962D27037EE693BDF096CC000E1A93332EEBBDECB9BDE749D3
:20E4E000962D27037EE693BDF096CC00171A93332EEBBDEC5118CE0064BD9C33CCC179DD66
:20E5000058142980BDE749962D27037EE69318CE0190BD9C33BDECDBBDF096CC001B1A93B7
:20E52000332EE14F91302703BDEC73BDE749962D27037EE693BDF096CC001BD3311A933364
:20E540002EE9BDECEFBDE749962D27037EE693BDF096CC001BD331D3641A93332EE71528A4
:20E5600080BDECB9BDEE8C2615BD9C73CCC1C0BDF042152980BD9C73CCC15FBDF042BDE736
:20E5800049962D27037EE6937A002F7A002FBDEE8C270220087C002F7C002F20E17C002F72
:20E5A0007C002FBDEC8118CE01F4BD9C33BDEC69142880CCC183DD58142980BDE749962D9F
:20E5C00027037EE693DC62C3001BD331D3641A93332EE8BDECDBBD9C5518CE01F4BD9C3334
:20E5E000BDECFD18CE01F4BD9C33BDED04DC141A8300002725CCC000DD58BDEC62BDE749CE
:20E60000962D27037EE693DC62C30028D331D364D3141A93332EE6BDECD4960381012727F1
:20E62000152880152980BD9C73CCC1C0BDF042BD9C557F00337F0034142930152B80BDF169
:20E6400023BDEA4D7EE3CBBDF123BD9C73CCC1C0BDF042BD9C55152980BDEA4DBD9C681568
:20E6600029B0CCC179DD58CCC215BDF0421428807F00337F0034BDE749962D27037EE69302
:20E68000BDED102608CC02321A93332EE9BD9C687EE4578601912D26037EE3298602912DE3
:20E6A00026037EE3368607912D26037EE3CB860A912D26037EE2FD860B912D26037EF42D0F
:20E6C000860C912D26037EE0D6860D912D26037EF1D77EEC1B9620C6033DC3007E8FA60016
:20E6E000973008A60097579706C6B73DDD319612C6033DDD64D331DD5A9611C6033DDD623C
:20E70000D35ADD5A9613498102270BC6033DDD14D35ADD5A2005CC000020F3C30028DD5A6D
:20E7200039BD9C7EBD9C73CCC237BDF04218CE01F4BD9C33BD9C73CCC1C0BDF04218CE01F3
:20E74000F4BD9C33BDEB3620D8BDEFE71329200713291003BDEF5C1227801496018101260A
:20E760000EBDED462709142780BDEA4D15278013290126BDEE18261E860F91422E1BBD9C8C
:20E780007E152930CCC259BDF0428605BDF3E5152901BDE721397F0042BDED322747BDEDA5
:20E7A000102749122A014C142A10860A91382E50BDEB64BDEB36142A01BDEB36152980BDA9
:20E7C000ED32260315290C142930BD9C68BDEA4D86009700152A01132901058607972D395C
:20E7E0008601972D39BDED6C270920B2BDED0B270920B0BDEDA2270220A4152A107F003889
:20E80000BDEDA22723BDED5A271E142A20860091392E1BBDED04BD9C73CCC26ABDF042863B
:20E8200006BDF3E5BDEB8C39152A207F00397A002EBDEE18271FBDEE50261A7C002E7A00A9
:20E840002E7A002EBDEE50261BBDEC3518CE00FABD9C33200F7C002EBDEC8F18CE00FABDAE
:20E860009C3320067C002E7C002E7A002FBDEDE0271FBDEE8C261A7C002F7A002F7A002F62
:20E88000BDEE8C261BBDEC3C18CE00FABD9C33200F7C002FBDECA418CE00FABD9C332006F6
:20E8A0007C002F7C002FBDED322720BDED72271B142A40865B913A2E18BD9C7ECCC27BBD74
:20E8C000F0428607BDF3E5BDEA9A39152A407F003ABDED8A2720BDED3E271B122A0817141E
:20E8E0002A08BD9C68CCC28CDD49BDF0428608BDF3E5BDEBB139122A043BBDED382607BDFA
:20E90000ED66261C2007BDED6627152000BDED202607BDED602609201CBDED6027022015FB
:20E92000142A04BD9C68CCC29DBDF0428609BDF3E5BDEBB1392056122B085213290212BDEA
:20E94000EDE0260D142A80CC044C1A933B2E11201A152A807F003B122A0227BDECDB202DCD
:20E96000BDEC697F0054142A022022BDECDBBD9C68CCC2AEDD49BDF042860ABDF3E5BDEBCD
:20E98000B139860691542E05152A0220CEBDED6C270B863D91362E0BBDECAB20067F003680
:20E9A0007F002D397F003DBDE749962D270139BDEDE0270ABDEDA82641BDECDB2005BDECDF
:20E9C0006920E4BDEDA82632BDEE502625BDE749962D2701397A002F7A002FBDEE8C270910
:20E9E0007C002F7C002F7EE9F27C002F7C002F7EE9C37F0037BDEDA82708BDECDB86009710
:20EA00002D39BDE749962D270139BDEC699637815B2E037EEA02BDECDB7C003D7EEA1F86DF
:20EA20000A913D2E25BDEE18270B8619913D2E1ABDEDA82615BD9C7ECCC204BDF042860294
:20EA4000BDF3E5152B08BDEBC8397EE9C31329200713291003BDEF5CBDE749962D2701393B
:20EA6000122904E9122908E57F0035BDE749962D7F002D270139BDED46260BBDECB28601D2
:20EA800097017F002D39BDECABBDEC4A860691352ED9866E91352ED32009BDEB36BDEB648B
:20EAA0007EE721BDEB36BD9C7ECCC226BDF0428603BDF3E520E4B6102D84F7B7102D398635
:20EAC000009701BDED322617BDEC4318CE07D0BD9C33BDE749962D270139BDED32272914FF
:20EAE00028807F0033BDED4C2729CC186A1A93332EF37F002D39BDE749962D270139862F7C
:20EB000091362EF27F002D39BDED4C2617864E91362EBFBD9C68CCC19EBDF0428601BDF35C
:20EB2000E57EEA9ABD9C73CCC248BDF0428604BDF3E5BDEBF039BDEC9DBDECEFBDECB9BD70
:20EB4000ECDBBDEC8FBDECA4BDECB2BDECABBDED04BDECD4BDECF6BDECFDBDECCDBDEC9695
:20EB6000152980397F00337F00347F003B7F003C7F003D7F003E7F00397F003B7F0027151E
:20EB8000288015293C152AF0152B0839BDEB64BDEB36BDEA4DBD9D8D122701F9122704F579
:20EBA000BD9C68122901058602972D398607972D39BDEB64BDEB36BDEA4D152903BD9C7E4E
:20EBC000DC49BDF0427EE721BDEB64BDEB36BDEA4D152933BD9C73CCC18DBDF042BD9D8D90
:20EBE000122701F9122704F5BD9C688601972D39BDEB64142A01BDEB36152A01BDEA4DBD51
:20EC00009D8D122701F9122704F5BD9C68122901058602972D398607972D39BD9C7ECCC0F1
:20EC20002CBDF0427EE721CE10081C000239CE10001C000839CE60001C000839CE60001CE6
:20EC4000000439CE60001C000239CE60001C000139CE10081C000414290439CE10081C00EC
:20EC60001039CE10081C000839CE10081C002014290839CE10001C008039CE10001C00407B
:20EC800039CE10001C002039CE10001C001039CE60001D000839CE10081D000239CE1000FD
:20ECA0001D000839CE60001D000439CE60001D000239CE60001D000139CE10081D0004124A
:20ECC0002A0109865B9741974014290439CE10081D001039CE10081D000839CE10081D0063
:20ECE00020122A0109865B9741974014290839CE10001D008039CE10001D004039CE10009A
:20ED00001D002039CE10001D001039962C840139962C840239962C84043984103984083923
:20ED2000B66002840439B66002840239B66002840139B6100A848039B6100A844039B610AD
:20ED40000A8420882039B61000840439B610008402880239B61000840139B66002848039B5
:20ED6000B66000840839B66000840439B66000840239B66000840139B61000844039B610AF
:20ED800000842039B61000840839B61008840439B61008841039B61008840839B6100884FC
:20EDA0002039B610008410398603B7103018CE0001BD9C33CE10301E008005860197233949
:20EDC0007F0023F6103486C43DCE0032028FCE000A028F17970691182E03860039860139C9
:20EDE0008602B7103018CE0001BD9C33CE10301E00800586019723397F0023F6103386C4D1
:20EE00003DCE0032028FCE000A028F17970691192E038600398601398604B7103018CE0046
:20EE200001BD9C33CE10301E00800586019723397F0023F6103186C43DCE0032028FCE005B
:20EE40000A028F17970691182E038600398601398600B7103018CE0001BD9C33CE10301EEE
:20EE600000800586019723397F0023F61031C02C86413DCE0095028FCE0001028F17800AD5
:20EE80009B66912E2E038600398601398601B7103018CE0001BD9C33CE10301E00800586DA
:20EEA000019723397F0023F61032C02C86413DCE0095028FCE0001028F17800A9B67912FDD
:20EEC0002E038600398601398600B7103018CE0001BD9C33CE10301E008005860197233967
:20EEE0007F0023F61031C02C86413DCE0095028FCE0001028FC00ADB66398601B71030181B
:20EF0000CE0001BD9C33CE10301E00800586019723397F0023F61032C02C86413DCE00953E
:20EF2000028FCE0001028FC00ADB673997737F0072BD9CAE8620BD9CFFCE0078A60081200E
:20EF40002704BD9C96390820F3DD72BD9CAE8620BD9CFFCE007820E4BD9C963913292079A8
:20EF6000BDED602704132B4017BD9C7E8681BD9C89BDEEC817BDEF2CCCC0FBBDF0422014FB
:20EF8000BD9C7E8681BD9C89CCC0F8BDF042CCC0F8BDF042BDED662704132B4014868BBD30
:20EFA0009C89BDEEFA17BDEF2CCCC0FBBDF0422011868BBD9C89CCC0F8BDF042CCC0F8BD4A
:20EFC000F042132B80148687BD9C89CCC111BDF0429620BDEF2C152910398687BD9C89CCE1
:20EFE000C0F8BDF04220EF13298056BD9C73DC58BDF042DC5A93330C59490C59490C594954
:20F000000C59490C5949CE0064028FDD5CCE003C028FD75E863C3DDD5FDC5C935FD7619695
:20F020005EBDEF2CCCC0E1BDF042966181092E06CCC115BDF0429661BDEF2CCCC0DDBDF013
:20F04000423983C000D3458FBD9C96393C183C3637BD9C73CCC117BDF042200CC61086102F
:20F060004A26FD5A26F82005BDED1027FB3332183838393C183C3736BD9C68CCC117BDF075
:20F08000423233183838393C183C3736BDED1027FB323318383839BD9C7EBD9C739633BDE0
:20F0A000EF49398600CEB709BD9D5A8600CEB70908BD9D5A8600CEB711BD9D5A8600CEB76C
:20F0C0001108BD9D5A8600CEB713BD9D5A8600CEB716BD9D5A8600BDF3E58600BDF3E58600
:20F0E00000BDF3E58600BDF3E58600BDF3E58600BDF3E58600BDF3E58600BDF3E58600BDB1
:20F10000F3E58600BDF3E58603CEB721BD9D5A8608CEB722BD9D5ABD9C68CCC0AEBDF04246
:20F120007EF120B6B716971FFCB709DD1AFCB711DD1CB6B713971E9B57813B2E56971EDC9F
:20F140001AC30001DD1A961F9B12813B2E02200C803C971F961E8B01971E961F971F961EDA
:20F16000CEB713BD9D5A961FCEB716BD9D5ADC1CCEB711BD9D5ADC1C17CEB71108BD9D5A9C
:20F18000DC1ACEB709BD9D5ADC1A17CEB70908BD9D5A39803C971EDC1CC30001DD1C209FC2
:20F1A000DD49BD9C7EDC49BDF042960781092E06CCC113BDF0429607BDEF2CBD9D8D1227BF
:20F1C000021296078B01970781142E0220D48601970720CE960739152940BDF9EEBD9C7EB9
:20F1E000BD9C73CCC0F8BDF042BDED0B2708CCC0E5BDF0422003BDF2E8BDED102708CCC05D
:20F20000E5BDF0422003BDF2E8BDED152708CCC0E5BDF0422003BDF2E8BDED262708CCC0CD
:20F22000E5BDF0422003BDF2E8BDED2C2708CCC0E5BDF0422003BDF2E8BDED322708CCC08A
:20F24000E5BDF0422003BDF2E8BDED382708CCC0E5BDF0422003BDF2E8BDED3E2708CCC052
:20F26000E5BDF0422003BDF2E8BDED462708CCC0E5BDF0422003BDF2E8BDED4C2708CCC016
:20F28000E5BDF0422003BDF2E8BDED542708CCC0E5BDF0422003BDF2E88681BD9C89BDED06
:20F2A000A89606BDEF2CCCC113BDF0428687BD9C89BDEDE09606BDEF2CCCC113BDF04286A1
:20F2C0008DBD9C89BDEE189606BDEF2CCCC113BDF042BDED1026037EF1DDBDED1026FBBD32
:20F2E0009C687E996F7EF2DACCC115BDF042397EF3A99617970486099705BDF3D726F096B0
:20F3000010970486099705BDF3D726E3960F9704865A9705BDF3D726D6960E9704864697A6
:20F3200005BDF3D726C996129704863C9705BDF3D7267696129704863C9705BDF3D72669D7
:20F3400096119704863C9705BDF3D7265C96189704865A9705BDF3D7264F96199704865A19
:20F360009705BDF3D7264296139704865A9705BDF3D726359616970486019705BDF3D72649
:20F38000289666970486149705BDF3D7261B9667970486149705BDF3D7260E96029704866E
:20F3A000159705BDF3D7260139BDF9A2860A97669767BDF8AD9666CEB714BD9D5A9667CE5C
:20F3C000B715BD9D5A86039717CEB706BD9D5A8662BDF3E57EE72196049105220220038637
:20F3E0000139860039CEB7E0E600BD9D5A0817E600BD9D5A0817E600BD9D5A0817E600BDE1
:20F400009D5A0817E600BD9D5A0817E600BD9D5A0817E600BD9D5A0817E600BD9D5A0817F2
:20F42000E600BD9D5A0817E600BD9D5A39BD9C73CCC2BFBDF042BDF9EE1529027F000DBD0B
:20F440009C7EBDF6D9BD9D8D12270208BDF6E8BDF83E20D9BDF83EBD9C73CCC2BFBDF0425A
:20F46000BD9C7ECCC2D0BDF042BD9D8D1227011E1227041ABD9C7ECCC2E1BDF042BD9D8DB6
:20F480001227010A12270406BDF9A27EF5EA7C000DBD9C7ECCC1C0BDF042BD9C7ECCC2E14E
:20F4A000DD47BDF606BD9D8D12270205BDF6E820E086019720BD9C7ECCC111BDF042962055
:20F4C000BDEF2C8603D6203DC3007EC30000DD098FA60081FF26048600A70081002708CC26
:20F4E000C103BDF0422006CCC10ABDF042CCC170BDF042BD9D8D12270210DE096C008602B4
:20F50000A10026026F00DF0920ABBD9C7ECCC111BDF0429620BDEF2CCCC303BDF042860304
:20F52000D6203DC3007EC30001DD098FA60081FF26048601A700BDEF2CCCC0FFBDF042BD91
:20F540009D8D12270210DE096C008609A1002ABA8601A70020B47C002096108B0191202727
:20F56000037EF4B57C000DBD9C68BD9C73CCC2BFBDF042BD9C7ECCC314BDF042BD9D8D12AD
:20F5800027016712270463BD9C7ECCC1C0BDF042BD9C7ECCC303DD47BDF606BD9D8D1227C3
:20F5A0000205BDF6E820E97C000D8609910D2AD77F000DBD9C7ECCC00ABDF042BD9C73CC69
:20F5C000C2BFBDF042BD9D8D12270107122704037EE0D6BD9C7ECCC3ADBDF042BD9D8D1224
:20F5E0002702078602970D7EF590BD9C7ECCC3BEBDF042BD9D8D122702037EF42DBDF8AD73
:20F60000BD9C687EE2FDBD9C73CCC2BFBDF042BD9C7E8611D60D3DD347BDF0428601910D08
:20F6200026059610BDEF2C8602910D260B960FBDEF2CCCC0FBBDF0428603910D260B960EDB
:20F64000BDEF2CCCC0FBBDF0428604910D260B9612BDEF2CCCC04EBDF0428605910D260B60
:20F660009611BDEF2CCCC04EBDF0428606910D26119618BDEF2CCCC117BDF042CCC0F8BD87
:20F68000F0428607910D26119619BDEF2CCCC117BDF042CCC0F8BDF0428608910D26219640
:20F6A000134981022712BDEF2CCCC04EBDF042CCC0F8BDF0427EF6C0CCC115BDF04220E950
:20F6C0008609910D261296162708CCC103BDF0422006CCC10ABDF04239BD9C7E8611D6172B
:20F6E0003DC3C3DFBDF042398600910D26127C0017BDF83E860991172A6F7F00177EF83A48
:20F700008601910D26107C0010860991102A5A860197107EF83A8602910D26237F0044CC72
:20F72000FF008FD6443AA600810026067F00447F000F910F2E057C004420E4970F202A8636
:20F7400003910D26277F0044CCFF158FD6443AA600810026067F00447F000E910E2E057C44
:20F76000004420E4970E7EF83A7EF83A8604910D26247F0044CCFF288FD6443AA60081000A
:20F7800026067F00127F004491122E057C004420E497127EF83A8605910D26237F0044CCF5
:20F7A000FF2F8FD6443AA600810026067F00447F001191112E057C004420E49711207B8630
:20F7C00006910D261296188B0A9718866391182A697F00187EF83A8607910D261296198B52
:20F7E0000A9719866391192A517F00197EF83A8608910D26237F0044CCFF3B8FD6443AA632
:20F800000081FF26067F00447F001391132E057C004420E4971320228609910D260F961652
:20F8200027057F0016201386019716200DCCC02CBDF04218CE03E8BD9C33BDF9E4399617EF
:20F8400081002607CCC4A0DD45202181012607CCC940DD45201681022607CCCDE0DD452020
:20F860000B81032607CCC000DD45204081042607CCD280DD45203581052607CCD710DD45EF
:20F88000202A81062607CC8DE0DD45201F81072607CC8000DD45201481082607CC84A0DDF6
:20F8A00045200981092605CC8940DD45399602CEB6D0BD9D5A960ECEB700BD9D5A960FCE45
:20F8C000B701BD9D5A9610CEB702BD9D5A9611CEB703BD9D5A9612CEB705BD9D5A9617CE97
:20F8E000B706BD9D5A9618CEB707BD9D5A9619CEB717BD9D5A9613CEB719BD9D5A9616CE35
:20F90000B720BD9D5A961ACEB709BD9D5A961CCEB711BD9D5ABDF9E4C600CEB60018CE00A4
:20F920007E18A600BD9D5A0818085CD12226F239B6B700970EB6B701970FB6B7029710B61D
:20F94000B7039711B6B7059712B6B7069717B6B7079718B6B7179719B6B7199713B6B720F5
:20F960009716FCB709DD1AFCB711DD1CB6B713971EB6B7149766B6B7159767B6B716971FFE
:20F98000B6B6D09702BDF2F2BDF9E4C600CEB60018CE007EA60018A7000818085CD12226A7
:20F9A000F33986059702863C970E8655970F8603971086149711861E971286289718860A63
:20F9C00097198601971386009716BDF9E4C600CEFF4818CE007EA60018A7000818085CD180
:20F9E0002226F3398603D6103DCB03D7223918CE012CBD9C337F002B18CE1024181C004010
:16FA0000BDEB64152AFF152980142B40860097560E18CE00C83901
:209900008682BD9C89BDEEC84F1BBDEF2CCCC0FBBDF042CCC113BDF042868ABD9C89BDEE06
:20992000FA4F1BBDEF2CCCC0FBBDF042CCC113BDF042BD9C7386C2BD9C89BDEDA89606BD45
:20994000EF2CCCC113BDF04286C7BD9C89BDEDE09606BDEF2CCCC113BDF04286CCBD9C896D
:20996000BDEE189606BDEF2CCCC113BDF04239BD9900BD9A82BDEC2E18CE0190BD9C33BD22
:20998000EC9DBD9900BD9A82BDEC7318CE0190BD9C33BDECEFBD9900BD9A82BDEC7A18CE20
:2099A0000190BD9C33BDECF6BD9900BD9A82BDEC8118CE0190BD9C33BDECFDBD9900BD9A3C
:2099C00082BDEC3518CE0190BD9C33BDEC8FBD9900BD9A82BDEC3C18CE0190BD9C33BDEC2C
:2099E000A4BD9900BD9A82BDEC4A18CE0190BD9C33BDECB2BD9900BD9A82BDEC4318CE0141
:209A000090BD9C33BDECABBD9900BD9A82BDEC8818CE0190BD9C33BDED04BD9900BD9A8296
:209A2000BDEC6218CE0190BD9C33BDECD4BD9900BD9A82BDEC5118CE0190BD9C33BDECB90D
:209A4000BD9900BD9A82BDEC6918CE0190BD9C33BDECDBBD9900BD9A82BDEC5B18CE019094
:209A6000BD9C33BDECCDBD9900BD9A82BDEC2718CE0190BD9C33BDEC96BD9900BD9A827EF6
:209A8000996FBDED0B2606BDEC9D7E9A90BDEC2EBDED102606BDECEF7E9A9EBDEC73BDED1E
:209AA000152606BDECF67E9AACBDEC7ABDED262606BDECFD7E9ABABDEC81BDED2C2606BD82
:209AC000EC8F7E9AC8BDEC35BDED322606BDECA47E9AD6BDEC3CBDED382606BDECB27E9AA4
:209AE000E4BDEC4ABDED3E2606BDECAB7E9AF2BDEC43BDED462606BDED047E9B00BDEC881D
:209B0000BDED4C2606BDECD47E9B0EBDEC62BDED542604BDECB939BDEC5139BDEABFBDED6E
:209B20003227F8BD9C688600970BBDEC35BD9BD4BDEC8FBD9BCCBDEC3CBD9BD4BDECA4BD6A
:209B40009BCC7C000BBDEC4ABD9BD4BDECB2BD9BCCBDEC2EBD9BD4BDEC9DBD9BCCBDEC5112
:209B6000BD9BD4BDECB9BD9BCCBDEC5BBD9BD4BDECCDBD9BCCBDEC62BD9BD4BDECD4BD9B5D
:209B8000CCBDEC69BD9BD4BDECDBBD9BCCBDEC73BD9BD4BDECEFBD9BCCBDEC7ABD9BD4BD03
:209BA000ECF6BD9BCCBDEC81BD9BD4BDECFDBD9BCCBDEC88BD9BD4BDED04BD9BCCBDEC2780
:209BC000BD9BD4BDEC96BD9BCC7E9B2618CE03E8BD9C3339BD9C73CCC078BDF0427C000BDB
:209BE000960BBDEF2CCCC0F8BDF042BD9BF2BD9BCC39BDED0B2703142B01BDED10270314BB
:209C00002B01BDED152703142B01BDED262703142B01BDED2C2703142B01BDED4627031447
:209C20002B01BDED4C2603142B01BDED542703142B0139183C3CCE01470926FD38180926A7
:209C4000F4183839183C3CCE01470926FD38180926F418383986F0BDA25839371686ACBD17
:209C6000A25817BDA258333986A3BDA2588601BDA2583986A3BDA25886C0BDA2583986A31A
:209C8000BDA2588602BDA25839371686A3BDA25817BDA2583339A600270BBD9C5B088619FB
:209CA0004A26FD20F13918CE0014BD9C33397F006F7F00707F007186109775CE00718603F7
:209CC0009774A6009776840F80052B0696768B039776967684F080502B0696768B30977681
:209CE0009676A700097A007426D878007379007279007179007079006F7A007526BD39CE52
:209D00000078A700088C007C26F8CE0000966F840F27058B30977808967044444444260650
:209D2000D678C12027058B309779089670840F2606D679C12027058B30977A089671444471
:209D400044442606D67AC12027048B30977B9671840F8B30977C7F007D3937183CC616F72B
:209D6000103BE700C617F7103B18CE000ABD9C337F103BC602F7103BA700C603F7103B1878
:209D8000CE000ABD9C337F103B1838333936373C183C1527072025BDED0B26F9BDED1026A0
:209DA000F4BDED1526EF18CE0019BD9C33BDED0B26E3BDED1026DEBDED1526D91329400A90
:209DC000BDE749962D27037EE693BD9E3896008101272896008102270896008103273620D9
:209DE000DB18CE0002BD9C33142702142B0218CE015EBD9C3386009700203418CE0002BDAF
:209E00009C33142701142B0218CE015EBD9C3386009700201A18CE0002BD9C331427041407
:209E20002B0218CE015EBD9C33860097002000142B011838383332391329200713291003CF
:049E4000BDEF5C39DD
:20A00000BDA116BD9C6818CE012CBD9C338600970B9700BD9C7ECCC03DBDF042960BBDEFD1
:20A020002CBD9C73CCC2BFBDF042BD9D8D12270107122704037EA04B7C000B960B810A2741
:20A04000037EA0138600970B7EA013CC0000DD09BD9C7ECCC03DBDF042960BBDEF2CDC09D4
:20A06000BDEF49BD9C73CCC2BFBDF042BD9D8D12270107122704037EA092DC09C30001DD45
:20A08000091A83000A27037EA050CC0000DD097EA050960BB1B7212617960AB1B722261091
:20A0A0002007860C972D7EE693860B972D7EE693BD9C68960B8107260ADC091A830002261C
:20A0C000022007860A972D7EE6938600970BBD9C7ECCC03DBDF042960BBDEF2CBD9C73CC44
:20A0E000C2BFBDF042BD9D8D12270107122704037EA1067C000B960B810A27037EA0CE8614
:20A1000000970B7EA0CE960B810926B7BD9C68860D972D7EE693BDED1026FBBD9C7ECCC05C
:20A12000E7BDF042BD9C73CCC2BFBDF042CC0000DD33142880DC331A83000A2E05BDED0B0B
:20A1400027037EA0C3BDED1027EBB6B72127037EA003B6B72227037EA0037EA0A915294030
:20A16000BD9C68CCC11BBDF042B6B721BDEF2CB6B722BDEF2CBD9C73CCC2BFBDF042BD9D58
:20A180008D12270107122704037EA18F7EA225BD9C688600970BBD9C7ECCC03DBDF04296B0
:20A1A0000BBDEF2CBD9C73CCC2BFBDF042BD9D8D12270107122704037EA1CE7C000B960B37
:20A1C000810A27037EA1968600970B7EA196CC0000DD09BD9C7ECCC03DBDF042960BBDEFAA
:20A1E0002CDC09BDEF49BD9C73CCC2BFBDF042BD9D8D12270107122704037EA215DC09C30C
:20A200000001DD091A83000A27037EA1D3CC0000DD097EA1D3960BCEB721BD9D5A960ACE87
:20A22000B722BD9D5ABD9C68CCC12CBDF0427EA22E18CE6002181D00A0181C004018CE6003
:20A2400002181C0020393CCE10001C2D0C1C2B321D2B451C2D2038393C183CCE10001F2E65
:20A2600080FCB7102F183838393C3637CE1000B6102EF6102F8108271A81042722810227B9
:20A280002AC1C02732C1C62736C1C3273AC1CC273E2041864FBD9C5B8652BD9C5B203586AE
:20A2A0004EBD9C5B8645BD9C5B20298646BD9C5B8645BD9C5B201D142C01152C06201514C7
:18A2C0002C02152C05200D142C04152C032005152C0720003332383BF8
:008000017F
